:10000000831686018312860101308C00272882071F
:10001000A8345B34FA346B3446346B3454345B3478
:100020005E345134FC347A34FF34FF340000000075
:100030000000000000000000080016209A0B1D2898
:10004000080000009A0B21289B0B212808008C0334
:100050000C0807208F008C0A0C0807208D008E00EA
:10006000861716208D0B3028861316208E0B342809
:100070008F0B2E2886131D201D201D208C0A0C0896
:1000800007209000FF301006031948288C0A272803
:08009000212021202120042879
:00000001FF
